:020000040800F2
:10500000581A0020D5500008458C0008FB83000882
:105010000000000000000000000000000000000090
:10502000000000000000000000000000E5950008FE
:1050300000000000000000004D940008E196000808
:10504000E7500008E7500008E7500008E750000864
:10505000E7500008615B0008E7500008E7500008CF
:1050600000000000E7500008995A0008E7500008C7
:10507000E75000084588000800000000E7500008DD
:1050800000000000E75000080000000000000000E1
:10509000E750000800000000E7500008E750000853
:1050A000E7500008E7500008E75000085DA000083E
:1050B000E7500008E7500008000000000000000072
:1050C0000348854600F060FC004800475DAE0008DC
:1050D000581A00200448804704480047FEE7FEE7CE
:1050E000FEE7FEE7FEE7FEE77D970008C1500008F7
:1050F00030B50B46014600202022012409E00D4670
:10510000D5409D4205D31D469540491B25469540F7
:1051100040191546521E002DF1DC30BDF0B51FB40C
:105120000646002082B005464024019100901BE015
:10513000019922460F46304600F04EFB049A059B2B
:10514000801A994110D310461946224600F034FBCC
:10515000361A8F410197224601200021009F00F05E
:105160002BFB38184D4100902046641E0028DFDCE0
:10517000019B00982946324607B0F0BD03460B4319
:105180009B0703D009E008C9121F08C0042AFAD2FD
:1051900003E00B780370401C491C521EF9D2704783
:1051A000D2B201E00270401C491EFBD270470022BF
:1051B000F6E710B513460A4604461946FFF7F0FF16
:1051C000204610BD30B504460020034600E05B1CBD
:1051D000934203D2E05CCD5C401BF8D030BDF8B503
:1051E00002464A40D40F42004B0052085B089A42E4
:1051F00002D20246084611464A0023D0C30D4A0097
:10520000DDB2120EAD1A202D35DA49020126490A07
:10521000F6058A19002C00D0524220214F1B11465E
:10522000B9402A411018C20D9A4221D0002C17D043
:10523000012D08DCDA05801AD20F8019D207DBB203
:1052400000F0F6FAF8BDDA05801A012340001B06CB
:10525000C01880185A428018CA0F1043490007E04E
:105260004908C2071143DA05801A801940088018DE
:1052700000F0D6FAF8BD61000122511A001BF7E7D1
:105280000122D2075140AAE70122D2075040A6E7E7
:1052900070B502464A40D50F40004A00ED0740086D
:1052A0005208002814D0002A12D0C40DD30D410298
:1052B0000120C0055202490A520AE41A09181218BC
:1052C0007D34914201D3641C00E04900002C01DAD6
:1052D000002070BD0023914201D3891A0343400886
:1052E00049000028F7D100290AD0914202D10121BA
:1052F000C90705E0914201D2012101E00121C94322
:10530000E005C018401900F08BFA70BDF0B50746F3
:105310000846584087B0C00F049048000E46590018
:1053200040084908BC1A884105D2384631461E4615
:1053300017460B4602465800400810434CD0300D2B
:10534000039040055900400D490D0590401A029008
:10535000402872DA18030121000B09050843019067
:1053600004980092002805D00199524200208841FB
:1053700000920190029840210A1A0199009800F0C9
:105380001BFA05460C466B4607CB00F036FAC019EF
:105390007141039A0E0D0023D71756401A467A40E2
:1053A000164344D0049A002A2DD0029A012A039A67
:1053B00015DC1205C01A914101263605001C714109
:1053C000D20F059ED2070093019202962A462346E9
:1053D00000F074FA07B0F0BD38463146FAE716051A
:1053E000224A0F46B218C01AB74101210905001C14
:1053F0004F4100187F41114618187941E20F1043C0
:105400006D19644113E0E2076D0815436408C20793
:105410001443039A01261205C01A91413605001C57
:105420007141CE07400830434908C01851412A460F
:10543000234600F036FACDE7FFE70498012240004A
:10544000C117121A00238B4104983146C417381A29
:10545000A141EEE730B40124E407634030BC55E7D6
:1054600030B40124E407614030BC4FE70000E0FFA6
:10547000F0B51FB488B00B990998002448400999E9
:10548000C00F490049080991C0070B9900904900D5
:1054900049080B9109990898A64608431CD00B9916
:1054A0000A98084318D0099801244000420D48008A
:1054B000410D099824050003000B204309900B9827
:1054C0000003000B20430B9050181C494018002289
:1054D00001901446104605E0002001460DB0F0BDD5
:1054E000032801DA034600E003239C46C11A0AAEF2
:1054F0000AE05F0008ADED5B4F00F75B7D430027DE
:10550000AA187C41491C5B1E6145F2DD410004ABD9
:105510005A522104120C0A43240C401C0828DFDBD9
:10552000019802900099704601910090059B049AA1
:105530000799069800F0C2F9D0E700000DFCFFFFC4
:10554000F0B50C465C4085B0E40FE40703944C00D2
:1055500000266408590094464908024602962243F0
:1055600021D062460A431ED06200570D4A000E0346
:105570002303550D012402462C492405781B1B0BDF
:10558000360B401823432643614600901C46501AB0
:10559000B44103D30098401C009002E09218009898
:1055A0005B41002803DA0020014605B0F0BD002071
:1055B000012109050746864611E064461D46141B75
:1055C000B54106D36546521BB341744607430C43AD
:1055D000A646CD0740084908284392185B41054676
:1055E0000D43EAD11046184313D060461946504087
:1055F0007140084306D06046101AB34106D201221A
:10560000002306E000220123DB0702E00122D2434F
:105610005310009874460105381C6141029C039D9B
:105620000019694100F03DF9BFE70000FD030000EB
:10563000C217C10F504010B54018CA079623002169
:1056400000F0F6F810BD10B500229623114600F0C8
:10565000EFF810BD0EB5C217C10F5040CA07401871
:105660000021054B0293019200910A460B4600F07F
:1056700025F903B000BD0000330400000EB5054954
:105680000291002100910A460B46019100F016F9A3
:1056900003B000BD33040000410040020122400A73
:1056A000D205090E80187F2901DA0020704796295B
:1056B00003DC9622511AC8407047963988407047DB
:1056C00070B5CD0F4A0009030123090B1B051943CF
:1056D0000B4BED070024520D9A4201DA002070BDF9
:1056E000074B34339A4203DC9A1A00F075F802E053
:1056F0000449511888402C43F1D0404270BD00004D
:10570000FF030000CDFBFFFF4A0009030123090B43
:105710001B051943094B10B5520D9A4201DA0020BE
:1057200010BD064B34339A4203DC9A1A00F054F849
:1057300010BD03495118884010BD0000FF03000050
:10574000CDFBFFFFC20FD207400040080BD0C10DB8
:105750000723DB01C91840020905400A1143C208AA
:10576000400711437047002001467047CB0FDB070D
:10577000490010B5490802460A4307D00A0D07241C
:105780000903E401090B121B002A01DC002010BDF3
:10579000C900440F0C43C100E018D205801800F086
:1057A0003FF810BD0122D207002800DB101A0029A3
:1057B00000DB511A8142704710B5202A04DB0146F4
:1057C000203A9140002010BD914020239C1A0346AE
:1057D000E3401943904010BD10B5202A04DB084671
:1057E000203AD040002110BD0B46D340D0402024A9
:1057F000A21A91400843194610BD10B5202A06DBB5
:10580000CB170846203A1041C1170B4306E00B4660
:105810001341D0402024A21A91400843194610BDDC
:10582000002904DA401C490001D1400840007047BB
:1058300070B40024050C05D11024000402D1002905
:1058400021D01124050E01D100020834050F01D129
:105850000001241D850F01D18000A41C002801DB5C
:105860004000641C002908D020252E1B0D46F54061
:10587000A14000D001212943084301061B1B000A57
:10588000DB1D02D5002070BC7047DB05181880189E
:105890000029F8DA401C4900F5D170BC40084000EE
:1058A000704710B5002B08DA0024401C61419218A3
:1058B0005B411A4301D14008400010BDF0B51FB450
:1058C00082B005460C0003D0084604F085FC02E0D7
:1058D00004F082FC20300246009021462846FFF763
:1058E0006BFF049B059A04460F4618431143084377
:1058F00014D0184610431BD0009840210A1A1846AD
:105900000599FFF769FF05460E46009A0599049828
:10591000FFF752FF084305D0012004E02046394636
:1059200007B0F0BD0020C11705430E432C43374399
:1059300000990E986305401A7905E40A00220C4389
:10594000FD0A0A3002D500200146E9E701051019D9
:1059500069410C9C0D9D00196941FFF7A2FFDFE72B
:1059600010B5002904DB0124E40740428C412146A4
:10597000002B04DB1C460123DB075242A341994262
:1059800000D1904210BD0000064C0125064E05E0F6
:10599000E36807CC2B430C3C98471034B442F7D350
:1059A000FFF792FBDCB10008FCB1000838B50446F3
:1059B000074908480068FFF79BFB6043009002E03E
:1059C0000098401E009000980028F9D138BD0000D2
:1059D00040420F00EC00002070B50446002520680E
:1059E00080688007800F012807D120680068C00701
:1059F000C00F002801D0012000E00020002839D18C
:105A0000206880681C490840002801D1012000E07E
:105A10000020002809D1606D102108436065A06D49
:105A200001210843A065012070BD20688068012124
:105A30000843216888600120FFF7B8FF01F070F982
:105A400005460EE001F06CF9401B0A2809D9606D8B
:105A5000102108436065A06D01210843A065012065
:105A6000E2E720680068C007C00F012148404840B5
:105A70000028E7D00020D7E71700008010B50023EA
:105A80001A4603E0845CE3189BB2521C8A42F9D3A5
:105A9000D84380B210BD000010B5034800F03EFEB0
:105AA000024800F03BFE10BDF4150020AC150020AC
:105AB00030B51C25446C2C400125A540046C656064
:105AC000046863608468102C04D10468A2600468D0
:105AD000E16003E00468A1600468E26030BD00009A
:105AE00010490120487202205E31487203203C397F
:105AF000487204200E3948720A4B0B495A1C087828
:105B00005871497899712333187159712033187776
:105B10005977107551751A461E32107551751076E9
:105B20005176704720110020D800002010B503F0F6
:105B300031FD202003F0CAFD012004F015FF0020F4
:105B400003F0C4FD044804F0B3FD044805F05CF81C
:105B5000002005F091F810BDA8000020838000000F
:105B600070B505200121000701F0CAF800240D4D91
:105B7000002800D02C6002210B4801F0C1F8002859
:105B800008D10A482C6000880A2148430849088047
:105B900004F076FA012000F0ADFF022000F0AAFF29
:105BA00070BD0000E400002000040050CC00002084
:105BB000D60000207047000000210A4A51610A49BE
:105BC0004968012252021143074A5160114649684F
:105BD00008221143044A51600021C209D201116018
:105BE000704700003C160020002002407FB50025D1
:105BF0000C460646039500F035FFE009029003A924
:105C000001960095684600F0AFFE002804D000F031
:105C1000F1FE002004B070BD00F0ECFE0120F9E7B9
:105C200010B5002302E0C45CCC545B1C9342FAD351
:105C300010BD0000002039498969FF22013211405E
:105C4000914208D13649496902221143344A5161CF
:105C5000FF21013108433149896901225202114073
:105C6000914208D12E494969012211432C4A5161C0
:105C70000121490208432949896901229202114000
:105C8000914208D12649496908221143244A5161A9
:105C9000012189020843214989690122D202114068
:105CA000914208D11E494969042211431C4A51619D
:105CB0000121C9020843194989690122520311408F
:105CC000914208D11649496910221143144A516181
:105CD00001214903084311498969012252041140F5
:105CE000914207D10E494969202211430C4A516162
:105CF0002021084309498969012212041140914277
:105D000008D10749496940221143054A51610121DF
:105D100009040843014988617047000000200240DF
:105D20003C16002070B5044600F0FAFF05460BE073
:105D3000601C002808D0002C04D000F0F1FF401BAC
:105D4000A04201D9032070BD1F488069C007C00F61
:105D50000028EDD11C48806902210840022801D1A9
:105D60001949886118488069FF210131084088423B
:105D700023D0154880694900084088421DD0124848
:105D8000806949000840884217D00F48806949005F
:105D90000840884211D00C48806989000840884238
:105DA0000BD00948806909010840884205D006489F
:105DB000806949100840884203D1FFF73BFF01206A
:105DC000C1E70020BFE7000000200240F8B51746F9
:105DD000002605460C4600F045FE09E02946022053
:105DE000226800F017FE002804D1241D2D1D361D49
:105DF000BE42F3D300F0FEFDBE4201D20020F8BD4A
:105E00000120F8BD10B5084902460020054B49792C
:105E100005E044001C5B944203D0401CC0B28842A1
:105E2000F7D310BD621200204800002010B50948C9
:105E300001F054F980B2FFF721FC074A074BFFF746
:105E400017FB0022064BFFF77BFBFFF75DFC80B2E0
:105E500010BD0000A4140020F853E3A59B843E402D
:105E600000408F40F8B5404CE079002801D0002078
:105E700000E00120E0713C493C48CA790275097A8A
:105E800041753B490A7802764978417637490520C1
:105E900013314872962004F0A7FE4B20C00004F096
:105EA000BDFE3249002213310C2004F087FF00218F
:105EB0000C2004F095FF022004F0E6FE2D4D002199
:105EC0000F2004F00BFE2842E062F8D0E06A411C8B
:105ED0003BD0294E294F400439D58122D2010021DF
:105EE0000F2004F040FF0021102004F0F7FD4106D0
:105EF0001E48490E0022633004F026FE1B4D633518
:105F0000687A052820D102221949681DFFF75AF93D
:105F1000002819D1A87A607113480422691C403006
:105F2000FFF72CF9206C00F02DF86083607929468A
:105F300042000B3108467330FFF720F9608B31883F
:105F40004843388002202070F8BD02F0B9FE0C48AA
:105F50000188608B0546FFF7CBF8308841433980D4
:105F60006D1E6583F8BD00004800002081110020EF
:105F7000D800002000D02724C6000020C400002044
:105F8000C800002010B504460E4801F0A7F80E49DD
:105F9000C006C00E098805E02246C240D2070FD0D5
:105FA000401CC0B28842F7D3012005E02246C2401F
:105FB000D20705D0401CC0B28842F7D3491EC8B2F0
:105FC00010BD0000A4140020C800002010B508482F
:105FD00000F03AFB0A21064800F0C0FA044800F03D
:105FE0006FF9800503D5024800F06DF980B210BD4D
:105FF00048140020F8B52F4D00220121284600F05A
:1060000088FEFFF7E3FFFFF71EFB2B4E3146FFF73D
:106010003FF92A4C0122A0601146284600F079FE83
:106020002749A068002588423EDB2078254F0028BC
:1060300015D02570FFF7CAFFFFF705FB3146FFF7C4
:1060400027F9A060FFF77EFB00223B46FFF702FA2C
:1060500000221D4BFFF70CFAFFF788FB6060A06879
:10606000FFF770FB00223B46FFF7F4F9174A184B85
:10607000FFF7FEF906460F466068FFF763FB134A19
:10608000144B5242FFF7F4F932463B46FFF73EF914
:10609000FFF76CFB10496060884201DD616004E03D
:1060A000FF21C905C84200D365606068FFF7F4FAB4
:1060B000C0B2F8BD0004005000401B442400002082
:1060C0000000604000000C4000E064403333333394
:1060D00033B33040CCCCEC3F0000C842F8B50446A6
:1060E00000250026002700BF5020005D012801D1B7
:1060F0000220F8BD01215020015500BF20688068B2
:106100008007800F012806D1206800680840002819
:1061100001D0012000E00020002841D1606DFF2166
:10612000013188430221084360652068C068870701
:10613000BF0F2068C068800880002168C8602068A0
:1061400080680121C90708432168886000F0E8FDE4
:10615000064611E000F0E4FD801B0A280CD9606DB2
:106160000221884310210843606500BF00215020B0
:10617000015500BF0120BCE720688068C00FC00740
:106180000121C9078842E5D02068C06838432168EA
:10619000C860606D0221884301210843606504E006
:1061A000606D202108436065012500BF002150205B
:1061B000015500BF28469CE770B504460D4600BF58
:1061C0005020005D012801D1022070BD0121502026
:1061D000015500BF2068806804210840800800281D
:1061E0000AD0606D20210843606500BF0021502067
:1061F000015500BF0120E8E72D496868884229D091
:106200002068806A29684903490B0843216888622D
:1062100028684003400B274908400121890488422F
:1062200008D12548806849010843234988600A202D
:10623000FFF7BCFB28684003400B204908400121C0
:10624000490488422CD11C488068490108431A49F6
:10625000886025E02068806A29684903490B8843E3
:106260002168886228684003400B124908400121D8
:106270008904884205D110488068490188430E4945
:10628000886028684003400B0C49084001214904FC
:10629000884205D1084880684901884306498860DA
:1062A00000BF00215020015500BF00208DE70000F5
:1062B00001100000000004480027014000000244D3
:1062C0000146486D704701460868006C7047000041
:1062D00010B50446002C01D1012010BD606D0028CE
:1062E00006D1A065002150200155204600F00EF98E
:1062F000606D10210840102806D0206880680421B5
:106300000840800800280AD0606D102108436065AD
:1063100000BF00215020015500BF0120DDE7606D66
:10632000FF210131884302210843606520688068AD
:106330008007800F012807D120680068C007C00FC0
:10634000002801D0012000E0002000283AD100BF41
:10635000032189076068884207D049426068884203
:1063600003D04900606888420CD120680069800031
:106370008008216808612068006961680843216815
:10638000086112E0206800698000800821680861C7
:106390005C4880680F21890488435A498860084610
:1063A0008068616808435749886000BF2068C068FA
:1063B000182188432168C8602068C068A168084324
:1063C0002168C8604F4880680121490688434D49CB
:1063D000886008468068A18E49060843494988605C
:1063E00020688068012109070840002804D120683E
:1063F00080680843216888602068C0684249084076
:106400002168C8602169E068022901D1042100E007
:10641000002108432021095D490308432C21095D1F
:1064200049000843216B0843A16989030843E169D6
:10643000C90308432168C96808432168C860FF216F
:10644000C231606A884207D0A16A606A0843216845
:10645000C96808432168C8602120005D012813D164
:106460002020005D002807D12068C06801210904B0
:1064700008432168C86007E0606D2021084360651B
:10648000A06D01210843A065E06B012817D12068A9
:106490000069FF218900884321680861216C606CD4
:1064A0000843A16C08432168096908432168086111
:1064B0002068006901210843216808610BE0206819
:1064C0000069C007C00F002805D020680069400897
:1064D00040002168086120684069C008C000216848
:1064E000486120684069A16B084321684861002029
:1064F000A065606D0221884301210843606500208A
:10650000EBE60000002701401902FEFF10B586B03F
:10651000044614216846FEF74AFE0E492068884268
:1065200016D10D48416B421511434163C16A0122E6
:106530001143C162C06A6946104005900220009074
:1065400003200190002002900520000700F0E2FAED
:1065500006B010BD0024014000100240F8B504460A
:106560000D46002600276069082801D1082711E0A0
:106570002068C068C007C00F00280AD0606D2021C5
:106580000843606500BF00215020015500BF012075
:10659000F8BD0C2700F0C4FB064614E0681C002878
:1065A00011D0002D04D000F0BBFB801BA8420AD9FB
:1065B000606D04210843606500BF00215020015533
:1065C00000BF0320E4E72068006838400028E5D0D9
:1065D000606D01214902084360652068C06803219D
:1065E00089020840002826D12020005D002822D101
:1065F000206800680821084008281CD120688068AD
:1066000004210840800800280DD1206840680C2132
:10661000884321684860606DFF2101318843012172
:106620000843606507E0606D202108436065A06D48
:1066300001210843A065A069002802D10C2021682F
:1066400008600020A4E7000070B50446002520681B
:10665000806804210840800800282BD100BF50200A
:10666000005D012801D1022070BD0121502001559B
:1066700000BFE069012803D02046FFF7ADF90546C9
:10668000002D18D1606D0D490840FF2101310843EC
:1066900060650020A06500BF00215020015500BFAB
:1066A0001C20216808602068806804210843216854
:1066B000886000E002252846D6E70000FEF1FFFFD3
:1066C00070B5044600252520005D022803D0042073
:1066D000E063012520E0206800680E2188432168DE
:1066E00008602068006840084000216808601C219C
:1066F000606C084001218140206C4160012125200F
:10670000015500BF00212420015500BFA06B0028C7
:1067100002D02046A16B8847284670BD70B504465C
:10672000206C0568206806681C20616C014004200C
:106730008840284000281DD004203040002819D06F
:106740002068006820210840002805D120680068E2
:1067500004218843216808601C21606C08400421E2
:106760008140206C4160206B00285AD02046216B6C
:10677000884756E01C20616C014002208840284078
:10678000002825D002203040002821D02068006851
:1067900020210840002808D1206800680A21884389
:1067A000216808600121252001551C21606C0840EA
:1067B00002218140206C416000BF0021242001554E
:1067C00000BFE06A00282CD02046E16A884728E014
:1067D0001C20616C0140082088402840002820D0FF
:1067E0000820304000281CD0206800680E21884313
:1067F000216808601C21606C084001218140206CE8
:1068000041600120E06301212520015500BF0021E6
:106810002420015500BF606B002802D02046616B28
:10682000884770BD70B50446002C01D1012070BDB1
:10683000244A2168881A1421FEF75AFC80006064FB
:106840002048083820640221252001552068056869
:106850001D480540E168A068084321690843616953
:106860000843A1690843E1690843216A08430543D5
:106870002068056001218903A068884217D011486B
:106880007830806A1C22616C11400F228A4090434C
:106890000C49783188621C22616C11406068884024
:1068A00008497831896A08430649783188620020AE
:1068B000E0630121252001550021242001550020FD
:1068C000B5E70000080002400F80FFFFF8B504465E
:1068D0000D4616461F460020009000BF2420005D94
:1068E000012801D10220F8BD01212420015500BF5B
:1068F0002520005D01282DD10221252001550020F1
:10690000E0632068006840084000216808603B465A
:10691000324629462046FFF7CBF8206B002806D0E8
:10692000206800680E210843216808600BE0206899
:1069300000680421884321680860206800680A21F3
:106940000843216808602068006801210843216825
:10695000086006E000BF00212420015500BF02208E
:1069600000900098BFE70000F8B504460E460127E6
:10697000002500BF1C48007C012801D10220F8BD81
:1069800001201949087400BF1848FFF7CBF90746E2
:10699000002F22D1401E3060656817E02846FFF7BF
:1069A0000BF91248FFF7BEF9074611484068082165
:1069B00088430F49486008464068491588430C4998
:1069C0004860002F01D0356006E08035A068C00126
:1069D00061684018A842E1D800BF00BF002002490A
:1069E000087400BF3846CAE73C16002050C30000B8
:1069F00000200240064840680221084304494860DC
:106A0000084640680121084301494860002070475A
:106A100000200240F8B507460C461546012600BF87
:106A20000E48007C012801D10220F8BD01200B494D
:106A3000087400BF0A48FFF775F90646002E06D114
:106A40000649486125600648FFF76CF9064600BF15
:106A500000200249087400BF3046E6E73C160020DB
:106A600050C300001D484068C007C00F002816D062
:106A700000BFEFF31080014600BF72B61848174AF6
:106A8000D0601848D06000BF81F3108800BF104666
:106A90004068C007C00F002801D0012070470F4890
:106AA000406802221040022815D100BFEFF3108089
:106AB000014672B60C48094A10610C48106108463C
:106AC00080F3108800BF1046406802221040022860
:106AD00001D10120E2E70020E0E7000000200240B1
:106AE000EFCDAB8905040302BFAE9D8C16151413C0
:106AF0007047000010B50446054840692040002852
:106B000004D0034844612046FFF7F2FF10BD0000A7
:106B10000004014070B50346002200240020DAE0A2
:106B2000012696400D6835402C46002C77D04D68E4
:106B3000022D02D04D68122D15D1D508AE001D468C
:106B40002035A8595507EE0E0F25B5400646AE4331
:106B500030465607F60E0D69B5402843D508AD00FE
:106B60001E46203670514D68012D08D04D68022D0B
:106B700005D04D68112D02D04D68122D18D198689E
:106B800056000325B5400646AE4330465600CD6854
:106B9000B540284398605868012595400646AE43A5
:106BA000304610264D6835402D09954028435860E1
:106BB000186856000325B5400646AE4330460D79A9
:106BC000AD07AD0F5600B54028431860D868560091
:106BD0000325B5400646AE43304656008D68B540A5
:106BE0002843D860012636074D683540B54271D13B
:106BF0003C4D6D6B012635433A4E75633A4D960810
:106C0000B600A85995072E0F0F25B5400646AE438E
:106C1000304605252D07AB4202D1002515E059E08D
:106C2000324DAB4201D101250FE0314DAB4201D1D4
:106C300002250AE02F4DAB4201D1032505E02E4D80
:106C4000AB4201D1052500E006259607360FB54079
:106C50002843254D9608B600A851284D28680546BA
:106C6000A5432846012636044D683540B54202D179
:106C7000054625432846214D286068680546A543FA
:106C80002846012676044D683540B54202D10546B6
:106C900025432846194D6860A8680546A54328463F
:106CA000012636054D683540B54202D105462543DB
:106CB0002846124DA860E8680546A54328460126E7
:106CC00076054D683540B54202D105462543284634
:106CD0000A4DE860521C0D68D540002D00D01FE71A
:106CE00070BD000000100240080001400004005088
:106CF00000080050000C0050001C0050000401402F
:106D0000024613690B40002B01D0012000E0002057
:106D10007047002A01D0816100E081627047000065
:106D20000148006870470000E80000200248006841
:106D3000401C014908607047E800002010B500249D
:106D4000084800684021084306490860002000F018
:106D50000BF8002801D0012401E000F0F5F92046ED
:106D600010BD00000020024070B5044600257D21C2
:106D7000C90009480068FEF7BBF9064601F098F81B
:106D8000002801D0012504E000222146501E00F019
:106D9000FFF9284670BD0000EC00002070477047E6
:106DA000F8B52C4C01266078401C6070E670208B92
:106DB000401C2083208902F053FC274DE888FEF711
:106DC00042FC2649FEF764FA254F3968FEF707FAB8
:106DD000386002212348FFF793FF002809D00020E4
:106DE00020621F482049076820488F4212DD067044
:106DF00012E0E888FEF727FC1849FEF749FA216AF5
:106E0000FEF7EDF91A4920628842EADB1A4919486F
:106E1000C860E6E700210170688F401EFEF708FC9D
:106E20003946FEF7BFFC06D82079002803D0134866
:106E3000C1793143C171688FFEF705FC08490968C3
:106E4000FEF7B0FC04D22079002801D004F09AF8B3
:106E5000F8BD0000BC000020200D002000007A4496
:106E6000E400002000040050000040404E000020DC
:106E70000000A0400400FA0500ED00E0941100209D
:106E8000704710B50446002C01D1012010BD02212D
:106E90002E200155204601F0DDFC204600F0F4F8DC
:106EA00000212E20015500BF2D20015500BF0020DC
:106EB000ECE77047704710B5044620680068C007CB
:106EC000C00F01214840484000280CD0206880684D
:106ED000084048404840002805D00120216848600B
:106EE0002046FFF75DFF2068006802210840400847
:106EF00000280BD02068806808404008002805D092
:106F00000220216848602046FFF748FF206800689B
:106F100004210840800800280BD0206880680840C1
:106F20008008002805D0042021684860204600F031
:106F300009F92068006808210840C00800280BD023
:106F4000206880680840C008002805D00820216813
:106F500048602046FFF794FF206800681021084031
:106F6000000900280BD0206880680840000900282C
:106F700005D01020216848602046FFF710FF2068E8
:106F8000006820210840400900280BD02068806854
:106F900008404009002805D020202168486020468C
:106FA000FFF788FF2068006840210840800900281A
:106FB0000BD02068806808408009002805D0402058
:106FC000216848602046FFF774FF10BD70B5044685
:106FD000002C01D1012070BD6068012800D100BFE4
:106FE00026496069884200D000BF2E20005D00283D
:106FF00005D100212D200155204600F057F802212F
:107000002E2001552068C5686068012803D08905D5
:10701000A06A884203D11E212846884305461749A5
:107020006069884201D01648054016480540A168AD
:1070300060680843216A0843616A0843A16A0843FB
:1070400005436068012804D00121C905A06A88426F
:1070500003D1E16820690843054308496069884213
:1070600005D06169A0690843E169084305432068C8
:10707000C56001212E2001550020ACE7FFFF000074
:107080003F1FFFFFF8F119FF10B50068054988425E
:1070900007D10548816B4900490881630D2000F044
:1070A0005FF810BD007C00400010024010B5006881
:1070B000084988420CD10848816BC204114381639E
:1070C000002201210D2000F063F80D2000F054F89B
:1070D00010BD0000007C004000100240014608681E
:1070E000C069704710B5034602242E20C4541448CA
:1070F000006824072043124C20601868C0680124EF
:10710000E40420431C68E060186880680124204380
:107110001C68A06018680069012420431C68206175
:107120001868816118684261186800690424204366
:107130001C68206101242E20C454002010BD0000D2
:1071400000040140704700000448416B01221143D4
:107150004163816B02041143816370470010024058
:1071600000BFC206D20E01219140024A116000BF49
:107170007047000080E100E000BFC206D20E01218E
:107180009140024A116000BF7047000000E100E03A
:1071900070B504460D4616462946204601F054FDBA
:1071A00070BD0000024949688143014A516070473F
:1071B0000070004003480068FF2101310843014985
:1071C0000860704700700040024949680143014A65
:1071D0005160704700700040074800680221084372
:1071E000054908600548006904210843034908610E
:1071F00000BF00BF30BF70470070004000ED00E0EE
:1072000010B5024600200E4B186880088000034627
:10721000134318460A4B18600A4B1B690424234386
:10722000084C2361012901D130BF02E040BF20BFDB
:1072300020BF044B1B690424A343024C236110BDEF
:107240000070004000ED00E0F8B504462021206801
:10725000084020287CD120680840202800D100BFA9
:1072600000278148806B012109070840002805D1CB
:107270007D48806B08437C49886301277B48006810
:10728000FF2101310840002816D1784800680843E2
:1072900076490860FFF744FD064606E0FFF740FD2B
:1072A000801B642801D90320F8BD70480068FF21C5
:1072B000013108400028F1D06B4805680321090519
:1072C0000D4060680840A8420DD009116068084070
:1072D000884208D164480068012149040840884276
:1072E00001D10120E0E76048403000690321090432
:1072F00008400546002D3DD060680840A84239D0BE
:10730000202120680840202834D1574840300069A7
:107310000321090488430546534840300069012190
:10732000C9040843504940310861084600690121F9
:10733000C90488434C4940310861084605618015FD
:1073400028408915884215D1FFF7EAFC064608E077
:1073500039E0FFF7E5FC801B4549884201D903204D
:10736000A2E7414840300069012149020840400A33
:107370000028EED000BF00BF032109046068084068
:1073800088420AD13848006809018843032212055F
:107390006168114008433449086000BF32484030FA
:1073A0000069032212046168114008432E494031EC
:1073B000086100BF012F05D12B48806B89058843E8
:1073C0002949886300BF2078C007C00F002809D072
:1073D00025484030C06880088000A16808432249E1
:1073E0004031C860022120680840022809D11E48A7
:1073F0004030C0680C218843E16808431A49403195
:10740000C86004212068084004280AD1164840308A
:10741000C068032189028843216908431249403129
:10742000C86008212068084008280AD10E4840306A
:10743000C068032109038843616908430A49403150
:10744000C86080212068084080280AD10648403062
:10745000C068032189048843A16908430249403177
:10746000C860002020E700000010024000700040CB
:1074700088130000F8B504460D46002C01D1012008
:10748000F8BD79480068C007C00FA8420ED2764800
:1074900000684008400028437349086008460068B7
:1074A000C007C00FA84201D00120E9E702212068EF
:1074B0000840022807D16D48C068F0218843A168C0
:1074C00008436A49C8602078C007C00F00284CD024
:1074D0006068022809D16548006801214904084014
:1074E000400C002824D10120CAE76068032809D194
:1074F0005E480068012149060840400E002817D167
:107500000120BDE76068012808D1584800680421BF
:107510000840800800280BD10120B1E753480068DB
:10752000012149020840400A002801D10120A7E7B3
:107530004E48C06880088000616808434B49C860B5
:10754000FFF7EEFB0646606802280FD107E0FFF761
:10755000E7FB801B4649884201D9032090E7434856
:10756000C0680C2108400828F1D134E06068032885
:107570000FD107E0FFF7D4FB801B3D49884201D9BA
:1075800003207DE73948C0680C2108400C28F1D160
:1075900021E0606801280FD107E0FFF7C1FB801BE5
:1075A0003349884201D903206AE73048C0680C217A
:1075B00008400428F1D10EE007E0FFF7B1FB801B83
:1075C0002B49884201D903205AE72848C0680C217A
:1075D00008400028F1D124480068C007C00FA84225
:1075E0000ED9214800684008400028431E49086021
:1075F00008460068C007C00FA84201D001203FE73D
:10760000042120680840042808D11848C0680721D0
:1076100009028843E16808431449C86008212068CA
:107620000840082809D11148C0680721C9028843C9
:107630002169C90008430D49C86000F049F80B49A9
:10764000C968F022114009090A4A515CC8400A4938
:1076500008600020FFF788FB0746002F01D038465E
:107660000EE700200CE7000000200240001002405E
:1076700088130000BAB10008EC000020014800683F
:1076800070470000EC00002000B5FFF7F7FF054948
:10769000C968072212021140090A034A515CC84016
:1076A00000BD000000100240CAB1000800B5FFF79D
:1076B000E5FF0549C9680722D2021140C90A034AF9
:1076C000515CC84000BD000000100240CAB1000873
:1076D000FEB52E48C7680C203840002845D0042845
:1076E00004D008280CD00C283ED10BE027480068B5
:1076F00010210840002801D0254C00E0254C41E035
:10770000254C3FE00F2080043840800C23490E5C5C
:10771000032080053840800D401C01901B48C06844
:10772000012109040840002807D01B49714308467D
:107730000199FDF7DDFC054614E0144800681021AE
:107740000840002807D01249714308460199FDF707
:10775000CFFC054606E00F49714308460199FDF745
:10776000C7FC05462C460DE000BF084840680721CD
:1077700049030840400B00900098401C01218140C3
:10778000CC0300BF00BF2046FEBD00000010024039
:1077900000093D000024F40000127A00D2B1000874
:1077A000FEB50446002C01D10120FEBDF848C66894
:1077B0000C210E40C768012109040F402078C00742
:1077C000C00F002872D0082E04D00C2E0FD108460E
:1077D00087420CD1EE480068012149040840400C62
:1077E000002863D06068002860D10120DDE700BF79
:1077F000012109046068884205D1E5480068084312
:10780000E349086027E005210904606888420ED139
:10781000DF480068012189040843DD490860084603
:107820000068012109040843D949086013E0D848D9
:107830000068012109048843D549086008460068AA
:10784000012109040840009000BFD1480068890068
:107850008843CF49086000BF6068002813D0FFF755
:107860005FFA054606E0FFF75BFA401B642801D982
:1078700003209AE7C6480068012149040840400CEB
:107880000028F0D012E0FFF74BFA054606E0FFF7BC
:1078900047FA401B642801D9032086E7BC480068EA
:1078A000012149040840400C0028F0D10221206841
:1078B000084002287AD1E0680290042E03D00C2EF2
:1078C00034D1002F32D1B24800680421084080082A
:1078D000002804D00298002801D1012065E7AC48B7
:1078E00040681F2109028843216909020843A84909
:1078F0004860084600680921884302990843A44962
:107900000860FFF7E5FEA249C968F02211400909A5
:10791000A04A515CC840A04908600020FFF724FA43
:1079200001900198002841D001983EE70298002874
:1079300024D0974800680921884302990843944954
:107940000860FFF7EDF9054606E0FFF7E9F9401B8F
:10795000022801D9032028E78D4800680421084047
:1079600080080028F1D08A4840681F210902884316
:107970002169090208438649486017E08448006885
:107980004008400082490860FFF7CAF9054606E052
:10799000FFF7C6F9401B022801D9032005E77C4800
:1079A00000680421084080080028F1D110212068D7
:1079B0000840102867D1002E36D17548006849016B
:1079C0000840400A002804D0A069002801D1012005
:1079D000EBE66F484068072149038843216A084362
:1079E0006B494860084640680002000A217F09068A
:1079F000084367494860206A400B401C01218140D0
:107A0000C8036349C968F02211400909614A515C01
:107A1000C840614908600020FFF7A6F9019001986D
:107A200000284BD00198C0E6A06900282CD0584807
:107A30000068FF210131084355490860FFF770F9DC
:107A4000054606E0FFF76CF9401B022801D9032028
:107A5000ABE64F480068012149020840400A00286F
:107A6000F0D04B484068072149038843216A084306
:107A700047494860084640680002000A217F09061D
:107A800008434349486019E041480068FF2101313B
:107A900088433F490860FFF743F9054606E0FFF7D2
:107AA0003FF9401B022801D903207EE638480068D0
:107AB000012149020840400A0028F0D1082120682D
:107AC0000840082839D1606900281BD03048403070
:107AD0000069012108432E4940310861FFF720F970
:107AE000054606E0FFF71CF9401B022801D90320D8
:107AF0005BE6274840300069022108404008002822
:107B0000F0D01AE022484030006940084000204987
:107B100040310861FFF704F9054606E0FFF700F978
:107B2000401B022801D903203FE619484030006974
:107B30000221084040080028F0D1042120680840B4
:107B4000042879D1002000901148806B89060840F4
:107B5000002806D10E48806B08430D498863012038
:107B600000900E480068FF210131084000281ED116
:107B70000A480068084309490860FFF7D1F805463C
:107B80000EE0FFF7CDF8401B642809D903200CE66E
:107B900000100240BAB10008EC0000200070004064
:107BA00085480068FF21013108400028E9D000BF66
:107BB000FF210131A068884205D18048006908434F
:107BC0007E49086130E0A06800280DD17B4800693B
:107BD000FF21013188437949086108460069091588
:107BE0008843764908611FE005210902A0688842A0
:107BF0000DD1724800690121890208436F4908616B
:107C000008460069891508436C4908610CE06B4817
:107C10000069FF210131884368490861084600690D
:107C2000091588436549086100BFA068002815D080
:107C3000FFF776F8054608E031E0FFF771F8401BE2
:107C40005F49884201D90320AFE55C480069012102
:107C500049020840400A0028EFD013E0FFF760F81F
:107C6000054607E0FFF75CF8401B5549884201D9FB
:107C700003209AE551480069012149020840400A61
:107C80000028EFD10098012808D14C484038806B7B
:107C900001210907884349494039886300BF606A68
:107CA00000284CD00C2E69D0606A022848D1434885
:107CB000403800680121090688434049403908607E
:107CC000FFF72EF8054606E0FFF72AF8401B0228CA
:107CD00001D9032069E53948403800680121490687
:107CE0000840400E0028EFD1E16AA06A0843216BEA
:107CF000084332494039C968FD22120491430843C0
:107D00002E494039C8600846006801210906084329
:107D10002A4940390860FFF703F8054606E0FEF7F8
:107D2000FFFF401B022801D903203EE523484038CD
:107D30000068012149060840400E0028EFD038E0D5
:107D40001E48403800680121090688431B49403914
:107D50000860FEF7E5FF054606E0FEF7E1FF401B81
:107D6000022801D9032020E5144840380068012189
:107D700049060840400E0028EFD11AE0606A012849
:107D800000D112E50D484038C76801200004384092
:107D9000A16A88420BD10F2080043840E16A8842F2
:107DA00005D1032080053840216B884201D0012095
:107DB000FBE40020F9E400000070004040100240A5
:107DC0008813000010B50446002C01D1012010BD1D
:107DD000606A002800D100BF0021A1625120005D2F
:107DE000002804D150200155204600F035F802212A
:107DF00051200155206800684021884321680860AF
:107E0000A16860680843E168084321690843616923
:107E1000084301225202A16911400843E169084365
:107E2000216A0843A16A084321680860A069000C20
:107E300004210840616A0843216848602068C069DD
:107E4000910088432168C8610020606501215120AC
:107E500001550020BBE7000010B586B00446142190
:107E60006846FDF7A4F910492068884219D10F48E7
:107E7000416B821411434163C16A01221143C16203
:107E8000C06A002110400590E0200090022001907F
:107E90000320039002910491052069460007FEF734
:107EA00039FE06B010BD0000003001400010024055
:107EB00070B504462546681E0949884201D901204B
:107EC0000CE0681E074948610321081F00F0BCFE52
:107ED00000200449886107200861002070BD00006F
:107EE000FFFFFF0000E000E070477047FEB504466A
:107EF0002068C56920680668206887682807000F21
:107F00000190019800280ED12020284000280AD096
:107F100020203040002806D0206E002802D02046C5
:107F2000216E8847FEBD019800287DD0F807C00F5C
:107F3000002804D1FF20213030400028F5D0E80788
:107F4000C00F00280BD0FF2001303040002806D0A1
:107F5000012021680862E06F01210843E0670220E8
:107F6000284000280AD0F807C00F002806D00220B9
:107F700021680862E06F04210843E067042028407C
:107F800000280AD0F807C00F002806D00420216876
:107F90000862E06F02210843E067082028400028BB
:107FA0000ED020203040002803D1F807C00F002851
:107FB00006D0082021680862E06F08210843E067C6
:107FC000E06F002846D020202840002809D020203B
:107FD0003040002805D0206E002802D02046216EB7
:107FE0008847E06F00902068806840210840402862
:107FF00004D0082100980840002826D0204601F02F
:10800000ACFD2068806840210840402819D12068D4
:108010008068884321688860E06E00280DD025487C
:10802000E16E8863E06E00E015E0FEF749FB002892
:1080300010D0E06E816B88470CE02046FFF755FFBB
:1080400008E02046FFF751FF04E02046FFF74DFF10
:108050000020E06766E701200005284000280CD0DA
:10806000012080053840002807D001200005216844
:1080700008622046FFF738FF54E780202840002898
:108080000AD080203040002806D0606E002802D040
:108090002046616E884745E740202840002807D0E9
:1080A00040203040002803D0204601F068FD39E729
:1080B00000BF37E7999A000810B50446002C01D19B
:1080C000012010BDA069002800D000E000BF606F53
:1080D000002805D1002170200155204600F02CF821
:1080E000242060672068006840084000216808601C
:1080F000204601F08FFD012800D1E2E7606A0028E8
:1081000002D0204601F090FB206840680921C90296
:10811000884321684860206880682A218843216854
:1081200088602068006801210843216808602046B3
:1081300001F0F2FBC5E70000F0B587B00646142158
:108140006846FDF734F82C493068884251D12B48F5
:10815000416B0122920311434163C16A0122114321
:10816000C162C06A002510400590032040020090C3
:108170000220032701A9A1C104200490052069461B
:108180000007FEF7C7FC1F4C1D48A560E56081C4D1
:108190008027E560A7602020256160610002A06162
:1081A0001848083CFEF73EFB002801D0FDF702FD11
:1081B000F466A662144C124821461438206003204D
:1081C000606010200831A1C16561A561E5612046AC
:1081D0002562FEF727FB002801D0FDF7EBFCB46613
:1081E000002201211B20A662FEF7D2FF1B20FEF712
:1081F000C3FF07B0F0BD000000380140001002408E
:1082000030000240AC150020F415002070B5044683
:108210000D461646A06F202863D1002D01D0002EF8
:1082200001D1012070BD01210903A068884208D155
:108230002069002805D1E807C00F002801D00120DF
:10824000F0E700BF7020005D012801D10220E9E7BE
:1082500001217020015500BF65655820065300209C
:10826000E0672220A067E06E002820D01E48E16E63
:10827000C8621E48E16E08631D48E16E4863002035
:10828000E16E88632368194624313346626DE06EDF
:10829000FEF71CFB00280AD01020E06700BF002179
:1082A0007020015500BF202060670120BAE700BFA1
:1082B00000217020015500BF20680068FF210131B6
:1082C000084321680860206880680121084321680C
:1082D0008860206880684021084321688860002009
:1082E000A0E702209EE70000039B00084D9B0008CA
:1082F000B19A000870477047FFB583B004460D4639
:108300001746606F202875D1002D01D0002F02D1B3
:10831000012007B0F0BD01210903A068884208D1FF
:108320002069002805D1E807C00F002801D00120EE
:10833000EFE700BF7020005D012801D10220E8E7CF
:1083400001217020015500BF0020E06721206067F7
:10835000FEF7E6FC019050200753522007530121FD
:108360000903A068884205D12069002802D10026AF
:10837000029502E02E460020029021E0069800902F
:10838000002280212046019B01F032FE002801D00E
:108390000320BEE7002E09D102980088C005C00D59
:1083A000216888620298801C029003E0307821687E
:1083B0008862761C5220005B401E81B2522001531D
:1083C0005220005B0028D9D106980090002240215D
:1083D0002046019B01F00CFE002801D0032098E705
:1083E0002020606700BF00217020015500BF0020E1
:1083F0008FE7FFE702208CE77047FEE710B5052402
:108400002407002204212046FEF783FC00220821D5
:108410002046FEF77EFC0A2002F003F90122042127
:108420002046FEF776FC0A2002F0FBF80022042129
:108430002046FEF76EFC10BD10B50524240700226F
:1084400004212046FEF765FC012208212046FEF7A4
:1084500060FC0A2002F0E5F8012204212046FEF724
:1084600058FC0A2002F0DDF8002204212046FEF725
:1084700050FC10BDF8B500240526074625463607F2
:10848000002204213046FEF744FC0A2002F0C9F81D
:10849000012204213046FEF73CFC6006040E082150
:1084A0003046FEF72DFC002801D0641CE4B2052004
:1084B00002F0B7F86D1CEDB2082DE1D3002F03D008
:1084C000FFF79CFF2046F8BDFFF7B6FFFAE770B54F
:1084D000052605463607002204213046FEF719FC22
:1084E0000024E80901D0012200E0002208213046E2
:1084F000FEF70FFC6806050E0A2002F092F8012232
:1085000004213046FEF705FC0A2002F08AF800221A
:1085100004213046FEF7FDFB0A2002F082F8641CBD
:10852000E4B2082CDDD370BD10B505242407012268
:1085300008212046FEF7EDFB012204212046FEF72C
:10854000E8FB002208212046FEF7E3FB0A2002F0A8
:1085500068F8002204212046FEF7DBFB10BD10B5B1
:1085600005242407002204212046FEF7D2FB002226
:1085700008212046FEF7CDFB0A2002F052F8012226
:1085800004212046FEF7C5FB012208212046FEF704
:10859000C0FB0A2002F045F810BD70B505252D0777
:1085A0000024012208212846FEF7B3FB062002F032
:1085B00038F8012204212846FEF7ABFB062002F022
:1085C00030F807E0641CE4B2FA2C03D9FFF7C7FFC8
:1085D000012070BD08212846FEF792FB0028F1D14A
:1085E000002204212846FEF794FB002070BD000005
:1085F000F8B501F0C9F901F003FA47480068C0690D
:10860000464E474F800700D5FE60FDF70FFC4549F9
:10861000454C0A7801218902002A1DD0012A04D084
:10862000022A06D0032A08D116E0FF22F532904232
:1086300012D200222046FEF76CFB0121C9023A4803
:10864000FEF75EFB394C0025002826D0384805602F
:10865000A079002802D005E00122EBE70120A071FB
:1086600001F00EFD2078632806D9002208212E484B
:10867000FEF74FFB012205E0012208212A48FEF700
:1086800048FB002201210520C9030007FEF741FB3A
:10869000284CA08C012803D01CE0A5710022ECE737
:1086A00025486946088072B680212448FDF79EFA65
:1086B000002804D0022269462048FDF787FB62B6F5
:1086C0001FA001F079FDA58402F0F8FC642001F000
:1086D000A1FFFE60608C012809D1164865844038EE
:1086E000058002F0EBFC642001F094FFFE60208C1A
:1086F000012806D1258402F0E1FC642001F08AFF04
:10870000FE600C48124A40380188914202D1C0886C
:10871000002800D1FE60F8BD2C1500200400FA05E9
:1087200000ED00E05A00002000040050BC000020D2
:10873000E4000020600D0020AAAA0000384A0008CA
:10874000BDF8C8EBC9FDBCB6C4A3CABD0D0A000084
:10875000AA55000008B53721202000F06EF803214B
:10876000212000F06AF84021222000F066F808215C
:10877000232000F062F8AA21302000F05EF80A48B9
:1087800002210187322000F058F80121332000F047
:1087900054F85F21202000F050F8684600F006F8F9
:1087A0000A2001F03EFF08BD200D002010B5014653
:1087B0000F2000F021F8002800D0012010BD10B5D6
:1087C0000446FFF7B1FE3220FFF781FEFFF7E5FE1A
:1087D000E0B2FFF77CFEFFF7E0FEFFF7A5FE3320D7
:1087E000FFF775FEFFF7D9FE0020FFF743FE0446B2
:1087F000FFF7B5FE204610BD10B50C46FFF7DFFFB2
:108800002070012010BD70B50D460446FFF78CFEA8
:108810003220FFF75CFEFFF7C0FEE0B2FFF757FE25
:10882000FFF7BBFE2846FFF752FEFFF7B6FEFFF745
:1088300096FE0A2001F0F5FE70BD10B5FFF7E3FFCC
:10884000012010BD10B50248FEF735FB10BD000039
:10885000A4140020F0B585B004460020039072B641
:108860004F4920684018002806D14E48C0680321AF
:1088700089040840039000E000BF00BF20688068C2
:1088800002902068C0680190206845692068866968
:1088900043492068401800280DD142484038806A7A
:1088A000490508433F49403988620846806A4000CC
:1088B0004008886200E000BF00BF002D01D1002EFB
:1088C0005FD0374920684018002807D13548C06874
:1088D0000321890488433349C86000E000BF00BF1A
:1088E000002D1DD02068006901210843216808611E
:1088F00020684561FEF714FA074600BFFEF710FA3C
:10890000C01B00902068006808210840082804D097
:108910007D21C90000988842F0D90820216848606C
:10892000002E1DD0206800690121084321680861DC
:1089300020688661FEF7F4F9074600BFFEF7F0F9FC
:10894000C01B00902068006810210840102804D047
:108950007D21C90000988842F0D910202168486024
:108960000F4920684018002809D10E48C06803212B
:1089700089048843039908430A49C86000E000BF9E
:1089800000BF206800694008400021680861029823
:108990002168886001982168C86062B605B0F0BDA2
:1089A0000084FFBF401002401CB500211648009112
:1089B000144A01910260C16312054260816007227E
:1089C0008263012202610246C16020321170FF23DE
:1089D0005170C23343628162117301638161042269
:1089E00041634261C161FDF773FC08480090801348
:1089F000019069460448FDF7DFFB00210248FDF7BE
:108A00006DFB1CBD0024014048140020020000043E
:108A100008B50848016B012211430163006B012175
:108A20001040009000220A20FEF7B2FB0A20FEF759
:108A3000A3FB08BD00100240F0B587B014216846C2
:108A4000FCF7B5FB4C48C26A04210A43C262C26A01
:108A50000A400592C16A80273943C162C16A394020
:108A60000591C16A01252943C162C16A2940059166
:108A7000C16A02263143C162C06A2A46304005906D
:108A800005201C210007FEF744F901223B493C4820
:108A9000FEF73FF900223B493948FEF73AF99121A8
:108AA0000520002209020007FEF733F9364801903D
:108AB000002405206946009502940007FEF72AF875
:108AC0000320019005206946009602940007FEF7F6
:108AD00021F80C2000901120019003200390052024
:108AE000029469460007FEF715F810200090052053
:108AF00069460396019502940007FEF70BF81120D2
:108B0000019002946946009503941D48FEF702F80F
:108B10001E4801906946009602951948FDF7FAFF34
:108B20001B48009002946946019503941448FDF790
:108B3000F1FFE8026A4651C269461148FDF7EAFFB3
:108B4000912000020090052002946946019503944B
:108B50000007FDF7DFFF6946094800970295019479
:108B6000FDF7D8FF002201210520FEF711FB0520AB
:108B7000FEF702FB07B0F0BD001002400106000046
:108B80000004005008300000000011100000211007
:108B90000836000010B50F4C0D482060FF2005304E
:108BA00060600020A060E06020616061E061012100
:108BB000206249026062A161A0620720E062204653
:108BC000FFF700F92068016840221143016010BDE1
:108BD00000300140D414002000B585B0142168464F
:108BE000FCF7E5FA164815490160E12149024160A8
:108BF00000218160C160016181610C22C16142611B
:108C00000162302141620121090381634900C1638E
:108C1000FFF752FA0120800200900220019001200B
:108C20000290032003900420049005206946000769
:108C3000FDF770FF01F01EFA05B000BD00380140DD
:108C40002C1500207047000010B5002819DA1A4AC8
:108C500003071B0F083B9B089B00D2588307DC0EC1
:108C6000FF23A3409A438B071B0E8407E40EA34007
:108C70001A43114B0407240F083CA408A4001A51FE
:108C800018E00E4A03231B02D21883089B00D25817
:108C90008307DC0EFF23A3409A438B071B0E840738
:108CA000E40EA3401A43054B032424021B19840835
:108CB000A4001A5110BD00001CED00E000E100E02E
:108CC000BFF34F8F04490348C860BFF34F8F00BF05
:108CD000FDE700000400FA0500ED00E0F0B58FB0FC
:108CE000962001F081FF4B20C00001F097FFFF4C60
:108CF00000256570A07B0C2801D30B20A0730122F6
:108D0000052051020007FEF704F8A07B6073607134
:108D1000A570F748A574F74E007830710221F64827
:108D2000FDF7EEFF002862D00020A179F14E490046
:108D30000843F071A06AF070401CA062607931466F
:108D4000B0724200CE310846C338FCF717FA06204D
:108D50007072304613380290217F0175617F417532
:108D600060790022400031460D3002F027F860792A
:108D7000002140000D3002F033F8022001F084FFA2
:108D8000F5712574A57201202073E572DB48FEF7AA
:108D9000A5F920840646A5706079FCF76FFCD84AD7
:108DA000D84BFCF765FB01F0D1FB0022D64BFCF75A
:108DB000ADFAFCF7A9FC0006C10C881980B20121AC
:108DC000C9036084884201D3401A6084CF4860633D
:108DD000E078401CE070C948FEF780F9E083CC4899
:108DE0000C90C4484E300B901630019025E20120C3
:108DF0009BE7C248FEF772F9E083C64EC64F21E0FA
:108E0000A07A002813D001F0B0FE039988420ED951
:108E1000069988420BD201F07FFD2573099801F075
:108E2000DCFE012001F030FF2072A57211E0B34892
:108E3000FEF754F980B2E083618C884202D3C919ED
:108E4000884206D300210F2001F048FE3042E06244
:108E5000D6D0E06A411C1FD040047DD58122D201CA
:108E600000210F2001F07FFF0021102001F036FECD
:108E70004106A048490E002250300A9101F064FEDC
:108E8000002001F0CBFE002001F07DFE994850301B
:108E9000417A0729AAD101E0FFF712FF9548022283
:108EA0009E495530FCF78EF900289FD100273E4699
:108EB0000DA801F060FE04200DAA390E36020E4303
:108EC0003902175C0F43401EF7D5A764E6640027FC
:108ED0003E46104601F041FE04200DA93A0E36022E
:108EE00016433A020F5C1743401EF7D527656665A7
:108EF000A1786A46491CA1707E494D310E791677DA
:108F00004A7969464A770092607B00280BD101209C
:108F100020716A46938B774ACE3213806071029833
:108F200006750099417573486946CE3000888F8B6D
:108F3000B8427DD10B997A48098A01806D4826464E
:108F40004C30808A20836D48FEF7C8F8F083308B60
:108F5000FF30C33080B200E064E172493083884260
:108F60000CD9494240186E49308308886D4A401C2C
:108F700080B20B320880904200D30D806A490320F2
:108F800008700B98594A81891186C089664B5086B2
:108F9000903B326B1A601A46B03AD37C1F073F0FE2
:108FA000032F00D0B7741A09F274F57001274F4AE5
:108FB000B7729186D0867079FF2191314843594923
:108FC000326D593940180104C817736D891858411A
:108FD0000206080A104355490990401803901921C8
:108FE0000998890240180690099841084900080E1E
:108FF0000902B165F0653F48F36C0A30B26C01F0CC
:1090000015FF3C48736D1630326D01F00FFF394883
:10901000F36D1230B26D01F009FF3648082141723C
:1090200070790022800033491C3001F0C7FE00E057
:109030009CE07079002180001C3001F0D1FE2D49A8
:109040002A48F772042251314030FCF797F834482F
:10905000318B07887D20C00078434018B0630D90A5
:1090600033480078F073009029484038C088FCF7F6
:10907000EAFA05903846FCF7E6FA0599FCF708F994
:109080007F21C905FCF7ABF8FCF706FB81B2284845
:1090900001800098401E814201D10120F072B78406
:1090A0001420305EFCF7D6FA07910890F08BFCF79D
:1090B000E5FA204A204BFCF7DBF900910A900D9865
:1090C000FCF7C8FA009B0A9AFCF7C4F9079B089AB8
:1090D000FCF71CF9FCF7F4FAF0631848008800F07C
:1090E000BFFAF07C00287DD00C9929E048000020D0
:1090F000BC0000209411002000040050A4140020A3
:10910000666666666666E63F00000840A086010067
:10911000600D002000D02724983A0000D8000020DD
:10912000E0000020E70300002413002000AEFCFF55
:10913000D4000020F853E3A59B843E40C4000020E7
:109140000988814279D00C98E17C01801222B448D0
:109150000199FCF713F80822B149B248FCF70EF860
:10916000AF49B0480A220831303051E13846FCF7A7
:1091700049FE617B224688420CD30121117151794D
:109180004300491C5171A649CE39CF5202990E7540
:10919000009B4B75A24B03210C3B19540B99A24B1E
:1091A0008E891E868600C9899D4859869C38116B18
:1091B00003468151B03BD97CA27C0807000F904246
:1091C00002D9032800D0A174E07C2746002814D0DF
:1091D00002229649581DFBF7F5FF00280DD101200A
:1091E000387400E029E09249C8710A981638C2B272
:1091F0007A748B480199FBF7C1FF8D487B6D30185D
:1092000016303A6D01F012FE78790022800088490C
:109210001C3001F0D3FD7879002180001C3001F072
:10922000DFFD0AE0324600210F2001F09CFD207B8B
:10923000002802D0002001F0A6FCE18B608C814266
:1092400000D2D6E57B4A80188142FAD87A4A0021BA
:109250000F2001F088FDA0786071714800260C385D
:109260000078002812D1206CFCF78CFE074673486A
:1092700001883846FBF73CFF71487F1E0088414358
:1092800088B270490880678300F0EAF90020A07373
:10929000627B2179521820E0614B0C3B195C00295C
:1092A00019D0A57BB7006D1CA573303BD9515C4D1F
:1092B0004300CE3DBC46ED5A7700594B761CB63B79
:1092C000DD5385001A335D5967463033DD51603315
:1092D000491EF6B21954401CC0B28242DCD8A078B4
:1092E000032801D2A07BA0734F490022887B4873DA
:1092F0000390401E31E000212BE0494C8B006C3C78
:10930000E6581D1906956D68AE4220DDB646444EFE
:109310004C00B63E365B9700B446414E3C3EF65993
:1093200007963F4E6C3EF55035464A3D67197D889D
:109330004A3E355334467A341C197A366568F550FE
:10934000069B76465E6066467E80079E6660491C88
:10935000C9B28142D1DB521CD2B28242CBDB32484D
:1093600000214172039C2BE02D4B2D4ACE3B4F0038
:10937000B63AD25BDA531D468A0062351E46AD58B6
:109380003236B550304EB54218D01D469235AD58E4
:109390000A2D13D1457A0626AC4675431E461A3E61
:1093A000FB18AE191B88B3801D4B65469C3BD21839
:1093B0001388F380528832816D1C4572491CC9B2F2
:1093C000A142D1D3164A00211F4B9C3A8C00491C64
:1093D000C9B213510C29F9D3007C002805D01049DB
:1093E0000B7848788A78022B0ED0134A00218032FD
:1093F0000F2001F0B8FC01210520002249020007DE
:10940000FDF787FC0FB0F0BD064BC91C9B1F181859
:10941000FBF7B4FE01F052FE642001F0FBF83BE5DF
:1094200030130020260D002048000020D800002026
:1094300094110020983A000000D02724C800002092
:10944000C6000020C4000020FFFF0100704700009C
:10945000F8B535493348086001F0D0FDFF20334DA1
:1094600013306880E888002801D16420E880304803
:109470000178432901D943210170E98E01702D4CF7
:10948000E88F2071A88F6071A87AA070A8880090DA
:10949000E0612889FCF7F2F8274A284BFBF7E8FF40
:1094A00001F054F80022264BFBF730FFFCF72CF9B3
:1094B00086B26681EF8831463846FBF719FEA081F7
:1094C00001460098FBF714FE71438EB27D20C00068
:1094D00026817043FCF7D2F81A4A1B4BFCF730F890
:1094E000FCF712F9E0817D2066823946C000FBF767
:1094F000FFFD2082E08201202083FCF797FCA08200
:10950000E28912491248FDF7EDFD12A0E16900F071
:1095100053FEE98813A000F04FFE298916A000F041
:109520004BFEF8BDADA0000844000020200D002037
:1095300000000020BC000020666666666666E63FA6
:1095400000000840F853E3A59B843E40FF7F0000E5
:10955000A4140020B1EAC7A949443A202564202E6A
:109560000D0A0000CDA8D1B6BCE4B8F43A202564B9
:10957000206D732E0D0A0000B5A5B4CECDA8D1B6CE
:10958000BBF9D5BECAFDC1BF3A202564B8F62E0D81
:109590000A00000070B586B014216846FBF707FE8C
:1095A00001250F4EED03002229463046FDF7B1FBA1
:1095B00001200024019002946946009503943046EE
:1095C000FDF7A8FA032001900294694600950394E0
:1095D0003046FDF79FFA022001F01CF806B070BD7E
:1095E0000004005070470000F8B5044600206A46A9
:1095F0001080194D55222A70AA226A700322AA707F
:10960000661DEE702A716971144A49008918AC719F
:109610002246E81DFBF7B2FD002007E029186A4644
:109620008978128889186A461180401CB042F5DB9F
:10963000611DA81CFCF722FA014668460180291921
:109640000078C8716846407808722146093102489E
:1096500000F0AEFAF8BD0000E4130020200D002059
:1096600010B513490A8BCB8A9A4201D3D21A0A83C6
:10967000104A098BD2884A437D211018C9004843FB
:109680000D490968401AFBF7E5FF0C4A0C4BFBF744
:1096900057FFFCF715F80B49884201DD4A42801854
:1096A000002800DA401808490968486110BD000028
:1096B000BC000020200D002084000020F853E3A50A
:1096C0009B843E40FF7F0000A4140020034A1168E1
:1096D000382389B29943014311607047003001403B
:1096E00010B5FDF723FB10BD10B59AB034216846C4
:1096F000FBF75DFD14210DA8FBF759FD1C2112A8F5
:10970000FBF755FD1B4801680324E402A143C21482
:1097100089180160FDF74EFD17480169A1430161F9
:1097200006200090FF2001300290012003901020BD
:1097300004900220099040040B90000100240C903A
:109740000A946846FEF72CF80F200D9003200E9027
:109750000F941094012111940DA8FDF78BFE812028
:109760001290032080041890149412A8FDF76CFD49
:109770001AB010BD0070004040100240154800684B
:10978000FF2101310843134908600846C0681249A7
:1097900008401049C86008460068104908400D4953
:1097A00008600846806840084000886008460068F5
:1097B000012189048843074908600846C068FD21E3
:1097C000090488430349C86000200861044805492A
:1097D00088607047001002400C40FF88F6FFF6FEDC
:1097E0000050000800ED00E010B501F08BF90C4CC2
:1097F00001E001F087F9A042FBD10A480021C182B3
:109800000078002809D0012802D0022805D102E002
:10981000FCF728FB01E0FFF761FA01F065F810BDE5
:109820003001CADE48000020818CC907C90F002919
:1098300008D001684968012252049143826A1143A9
:10984000026851600222416A1140022907D1016871
:109850004968D2039143C26A1143026851600422ED
:10986000416A1140042907D10168496812049143F3
:10987000026B1143026851600822416A11400829B5
:1098800007D10168496812039143426B1143026892
:1098900051601022416A1140102907D1016889687E
:1098A00012029143826B1143026891602022416A47
:1098B0001140202907D10168896812029143C26BC7
:1098C0001143026891604022416A1140402915D13C
:1098D0000168496892039143026C11430268516028
:1098E00001221205016C914208D1016849680322E6
:1098F00052059143426C1143026851608022416AD3
:109900001140802907D10168496812039143826C94
:10991000114302685160704738B504460020E06783
:10992000FDF7FEF905462068006808210840082870
:109930000BD114482B46002289040090204600F0E9
:1099400057FB002801D0032038BD2068006804219F
:10995000084004280BD10B482B4600220905009033
:10996000204600F045FB002801D00320ECE7202032
:109970006067A06700BF00217020015500BF002074
:10998000E2E70000FFFFFF01F8B5184CC826E078B9
:10999000002829D16079002826D101206071144D5A
:1099A000686B002700281ED0686BC821081A15E0D4
:1099B0001048E168405C616988470F480A210088C7
:1099C00048430E490880E068401CE060E068C82811
:1099D00000DBE760696BC820401A761EE1688142AF
:1099E00001D0002EE4DC6771F8BD000030000020DB
:1099F00000000240580C0020CC000020D6000020BF
:109A000070B5224CE07800283FD1207900283CD165
:109A1000012020711E4EF16900250906002933DA64
:109A20002156625791420AD1F06940062CD5A0799F
:109A3000002829D0A5712089401C208124E0A1792B
:109A4000002903D1A0710A2000F0EBFD0020205670
:109A5000CC2148430F494218206912181279B2628A
:109A6000401C00222061A256CC235A4389588142CF
:109A70000ADC25612078401C207020780E2800D157
:109A80002570A078401CA070257170BD30000020AA
:109A9000003801403001002070B50546AC6A002155
:109AA0005A200153522001532046FEF71EFA70BD82
:109AB000F8B50546AC6A666FA76F2068806880219C
:109AC0000840802807D1212E05D1002152200153C2
:109AD000204600F064F82068806840210840402853
:109AE00007D1222F05D100215A200153204600F032
:109AF00034F8E06F10210843E0672046FEF7F5F9DF
:109B0000F8BD70B50546AC6A286800682021084099
:109B1000002817D100215A20015320680068FF2136
:109B2000013188432168086020688068400840004F
:109B300021688860206880684021884321688860A7
:109B40002020A0672046FEF7D5FB70BD70B5044607
:109B5000A56A2846FEF7CFFB70BD01680968FF22A1
:109B600021329143026811600168896849084900FF
:109B7000026891602021816700210166704710B55D
:109B8000044620680068402188432168086020203E
:109B90006067002060662046FEF72EFC10BD01685D
:109BA0000968C02291430268116020214167704713
:109BB00070B5164CE278002A0CD12279002A09D11E
:109BC0000122E2700025C82903DC0222A256002AE5
:109BD00001DCE57070BD0123E356CC2253430C4AEF
:109BE000D1500123E356CC2673439B180A46014605
:109BF000181DFBF7C3FA6078401C607060780E286F
:109C000000D16570A078401EA070E2E7300000200F
:109C100030010020F0B587B00446102004900025E4
:109C2000002003900026E7492068884200D100E028
:109C300000BF2169A068084361690843E1690843DE
:109C4000074620680068E0490840384321680860FA
:109C500020684068032109038843E16808432168BC
:109C60004860A769D7492068884201D0206A074325
:109C7000206880680B210902884338432168886086
:109C800000BFD249206888421CD1D148C0688007F3
:109C9000800F002806D001280AD0022805D003280A
:109CA0000CD108E0012004900BE00220049008E0B1
:109CB0000420049005E00820049002E010200490A5
:109CC00000BF46E0C349206888421CD1C048C06834
:109CD0000C210840002806D004280AD0082805D006
:109CE0000C280CD108E0002004900BE00220049026
:109CF00008E00420049005E00820049002E0102011
:109D0000049000BF25E0AF49206888421FD1B048C9
:109D1000C068032189020840002808D00121890277
:109D2000401A0AD0401A05D0401A0CD108E0002091
:109D300004900BE00220049008E00420049005E069
:109D40000820049002E01020049000BF01E01020E1
:109D5000049000BF9B492068884256D1049804288B
:109D60001AD004DC002807D002281CD108E00828FB
:109D700016D0102817D117E0FDF786FC064616E02E
:109D8000934840380068102108400009002801D09D
:109D9000914E00E0914E0AE0FDF79AFC064606E07F
:109DA0000126F60303E000BF0120039000BF00BFBF
:109DB000002E0AD0606841004018B04203D86068A5
:109DC0000003B04202D201200390F4E060680290E8
:109DD0003046FF21013100F016FA62685208002374
:109DE0008018594101910090029AFBF797F90546B6
:109DF00003200002854205D37948854202D82068B5
:109E0000C560D8E001200390D5E00121C903E069D5
:109E100088426FD1049804283CD006DC002809D081
:109E2000012813D002284AD11CE008283ED010286F
:109E300045D145E0FDF728FC40006168490840181D
:109E400002906168FBF754F985B23CE0FDF72EFC07
:109E5000400061684908401802906168FBF748F9C2
:109E600085B230E05A4840380068102108400009A7
:109E7000002807D061684A085A4BD018FBF738F918
:109E800085B206E061684A08574BD018FBF730F9F5
:109E900085B218E0FDF71CFC4000616849084018D5
:109EA00002906168FBF724F985B20CE061684A080A
:109EB00001231B04D018FBF71BF985B203E000BF98
:109EC0000120039000BF00BF102D0FD347488542EB
:109ED0000CD846480F38284005902807400F0599B0
:109EE0000843059005982168C86064E0012003904C
:109EF00061E0FFE7049804283AD006DC002809D086
:109F0000012812D0022847D11AE008283BD0102897
:109F100042D142E0FDF7B8FB616849084018029061
:109F20006168FBF7E5F885B23AE0FDF7BFFB6168D1
:109F30004908401802906168FBF7DAF885B22FE013
:109F4000234840380068102108400009002807D045
:109F500061684A08204BD018FBF7CAF885B206E0C2
:109F600061684A081D4BD018FBF7C2F885B217E0AC
:109F7000FDF7AEFB61684908401802906168FBF785
:109F8000B7F885B20CE061684A080123DB03D018FA
:109F9000FBF7AEF885B203E000BF0120039000BFDD
:109FA00000BF102D05D31148854202D82068C56036
:109FB00001E001200390002020666066039807B04E
:109FC000F0BD000000480040F369FFEF0038014099
:109FD000401002400044004000093D000024F4000D
:109FE000FFFF0F0000127A000048E801FFFF0000A9
:109FF000FFB581B004460D4617460A9E22E0701C4C
:10A0000000281FD0FCF78CFE0499401AB04201D8FA
:10A01000002E17D120680068FF21A13188432168F4
:10A02000086020688068400840002168886020201F
:10A030006067A06700BF00217020015500BF0320AA
:10A0400005B0F0BD2068C0692840A84201D10120B8
:10A0500000E00020B842D2D00020F1E710B504495A
:10A060001020096808620248FDF740FF10BD00009B
:10A070002C15002001490D20887070473000002009
:10A0800010B507480A22018A51434183FEF7C0FCFC
:10A09000FEF7A2FDC82203490348FEF7B7F810BD3A
:10A0A000BC000020580C00202C150020F8B53D4CB9
:10A0B000002321783C4A1D46082910D0072945D0A5
:10A0C00006294ED0052950D0042951D0032952D059
:10A0D000002954D0012956D0022958D059E0A1783E
:10A0E00000264A1F04E0304FBF5DFB189BB2761C70
:10A0F0009642F8DB667927799A195118E3786278E5
:10A10000C9188918C9194018C0071AD0012E14D0CF
:10A11000022E16D125482449C018FBF72FF800F06D
:10A12000CDFF642000F076FABFF34F8F214920481D
:10A13000C860BFF34F8F00BFFDE759081046FFF717
:10A1400053FA2570E570A570A571F8BDA17950543A
:10A15000491CC8B2A071A178491F8842F5D10820D6
:10A1600001E0607007202070F8BDE0700620FAE77B
:10A1700060710520F7E7A070E5700420F3E755282B
:10A1800007D10120EFE7AA2803D10220EBE703283B
:10A1900003D02570E570A570F8BD032020702071F4
:10A1A000F8BD0000B300002080130020200D002027
:10A1B0000400FA0500ED00E00FB410B503A9044B4C
:10A1C000044A029800F01AF910BC08BC04B0184701
:10A1D00045AE0008F00000202021020C01D0102123
:10A1E0001046020A01D010460839020901D0104673
:10A1F000091F820801D01046891E420801D0881E1E
:10A200007047081A7047F8B582B28BB2040C0D0C77
:10A2100010465843002126465E43370C3604801909
:10A22000794116466E43370C36048019794126462B
:10A230006E438919F8BD30B47446641E2578641CD9
:10A24000AB4200D21D46635D5B00E31830BC18478B
:10A2500002E008C8121F08C1002AFAD170477047EF
:10A26000002001E001C1121F002AFBD1704708B590
:10A270000021684601706B46012202212C2000F06B
:10A2800081FD0221684601706B4601222C2000F0FE
:10A2900079FD08BD38B504466D20694608706B46E7
:10A2A000012207492E2000F06DFD0649002C01D047
:10A2B000054A00E0054A2E2000F04AFD38BD0000A6
:10A2C0000608000006180000070600000716000038
:10A2D00038B504466B4602220021362000F018FCF7
:10A2E000B3212300FFF7A7FF0E0F08153A3A3A3AB9
:10A2F0001C273A3A2F34483A0021684601704078CA
:10A300004108490014E06946087880088000401C34
:10A3100004E06946087880088000801C08701DE011
:10A32000684602780A404832027041788020014332
:10A330006846417012E0684602780A400270407830
:10A340004106490EF4E7694648780221084303E0D4
:10A3500069464878FD210840694648706B460122ED
:10A360000021362000F00EFD012200AB1146362000
:10A37000013300F007FD38BD69460878CF21084059
:10A3800069462030CAE708B50321684641700121BB
:10A3900001706B4602220021362000F0F3FC0122FE
:10A3A000D20306212D2000F0D3FC012000F032F969
:10A3B0000120FFF78DFF08BD08B5020A69464A7003
:10A3C00008706B46022204212D2000F0DBFC0320E4
:10A3D000694608706B46012206212D2000F0D2FC50
:10A3E0000020694608706B46012206212D2000F0EE
:10A3F000C9FC0A212D2000F071FB08BDFFB58DB00E
:10A400000446002506E025280AD0109A0F999047A7
:10A41000641C6D1C20780028F5D1284611B0F0BDD1
:10A4200000270121484A009700E00743641C237875
:10A430000846203B98401042F7D120782E2817D1AB
:10A44000042007436078641C2A280CD10E98641CF1
:10A4500002C800910E900BE000990A225143303956
:10A460004018641C00902078014630390929F3D93E
:10A4700020780028D1D0642808D0692806D0752813
:10A480001ED0109A0F9990476D1C5BE00A200E9920
:10A49000019001C90E91002802DA40422D2102E00C
:10A4A000390504D52B216A461172012103E0F90711
:10A4B00004D02021F7E70BAE0B910DE00021FAE765
:10A4C0000A200E99019001C90E91F7E70199FAF758
:10A4D0000FFE3031761E31700028F7D103A8801BA3
:10A4E00020300190780701D5009801E0012000900C
:10A4F0000199884201DD401A00E000200027009009
:10A5000006E002A8109AC05D0F9990476D1C7F1C51
:10A510000B988742F5DB04E0109A30200F999047A2
:10A520006D1C0099481E00900029F5DC05E030788C
:10A53000109A761C0F9990476D1C0199481E019046
:10A540000029F4DC641C65E709280100F8B54A001D
:10A550002B4B520DD6182B4A0C460546142E2BDADF
:10A56000002E12DA284BFAF7D1FE00221346FBF731
:10A57000F7F940D2002C03DA0124E40700253AE081
:10A580002046284337D0214C14E0214F0B46F7409A
:10A590003B402B4331D01C4BFAF7B8FE0022134648
:10A5A000FBF7DEF927D2002C03DD01200005F04087
:10A5B0000419BC4300251EE0332E1EDC3346002761
:10A5C000143BFF43DF40384217D00F4BFAF748FFE8
:10A5D00000221346FBF7C4F90DD2002C0ADD142E1D
:10A5E0000CD03420811B012088404019A84200D2A1
:10A5F000641C0546BD4321462846F8BD641CF9E7A6
:10A6000001FCFFFF9C7500883CE4377E0000F03FB2
:10A61000FFFF0F007D2110B5C900484300F001F88D
:10A6200010BD002140E000BF00BF00BF00BF00BF61
:10A6300000BF00BF00BF00BF00BF00BF00BF00BF22
:10A6400000BF00BF00BF00BF00BF00BF00BF00BF12
:10A6500000BF00BF00BF00BF00BF00BF00BF00BF02
:10A6600000BF00BF00BF00BF00BF00BF00BF00BFF2
:10A6700000BF00BF00BF00BF00BF00BF00BF00BFE2
:10A6800000BF00BF00BF00BF00BF00BF00BF00BFD2
:10A6900000BF00BF00BF00BF00BF00BF00BF00BFC2
:10A6A00000BF00BF00BF491C8142BCD370470000FF
:10A6B000FEB5044600200190009060797349400087
:10A6C0000E5A61782578491E7148CFB20163042D76
:10A6D00077D0072D75D000210291217801736C4944
:10A6E000E379012292058969002B6CD09143816145
:10A6F0006748217A4173217A82698907890B0A4365
:10A7000082610021042000F02EFB324661492E2098
:10A7100000F01EFB3846FFF7BDFD5F4E0522705D61
:10A72000810040185D49431807212B2000F02AFBC7
:10A730005B49029801220B180B21282000F022FB14
:10A74000705D584980000A580C21282000F00BFB4E
:10A75000E079554980004018A1794900425A022108
:10A76000272000F0F5FA51487E00825B0421272063
:10A7700000F0EEFAE079002829D0A07804282CD047
:10A7800028206946087220220621272000F0E0FADE
:10A7900002AB01222621272000F0F4FA44493801B7
:10A7A0004018E178890042580821272000F0DBFAA0
:10A7B000A17A601C627A0902114313D016E000E00E
:10A7C00001E0012188E71143F608816190E76422E6
:10A7D0000621272000F0BCFAE0E710206946087245
:10A7E0000246D1E733490172090A4172417A007A7F
:10A7F0000A0202432021272000F0AAFA2E4F0C2142
:10A8000023203A6800F0AFFAF0198288042123204F
:10A8100000F09EFAA07900280BD0E07927490122A8
:10A8200043180021212000F0ADFA032001900120FF
:10A8300000902A07120F1001024360780021800760
:10A84000000B0243019800050243009840040243B4
:10A850002079C006400902436079C00602431F20E8
:10A8600000F081FAA07861780123084302040848C7
:10A87000DB030261E179490319430A4302610021C4
:10A88000082000F070FA0020FEBD000088B100082A
:10A89000F40000200428000030B10008010000206E
:10A8A0001F00002038B1000858B1000864B100084A
:10A8B00068B100084110000050B1000821000020DC
:10A8C00038B50C4607498A8B002102432C2000F042
:10A8D0003FFA684604706B46012206212C2000F0E6
:10A8E00051FA38BDF400002010B5FFF7C0FC10BDD0
:10A8F00010B504460421362000F0F0F80121C90209
:10A90000002C01D0084300E0884302460421362091
:10A9100000F029FA10BD000038B5402069460870E3
:10A9200000210E2000F0DAF80446002211460E2025
:10A9300000F019FA6B46012200210D2000F022FAE6
:10A94000074A00210F2000F00EFA00F0E7F9224636
:10A9500000210E2000F007FA02480021017338BDE3
:10A96000F8FF2724140100207CB505460420694621
:10A9700008704B4C002060752146203120634871DF
:10A980000873A0836063A06300F0BCF8454E2060AC
:10A9900002E000F0B7F82060B042FAD10020FFF7E3
:10A9A00097FC41480078242801D9243806E0062184
:10A9B000FAF79EFB0622101A400108430206010422
:10A9C0000A4301020A43024300211E2000F0CBF992
:10A9D0006B4601220021242000F0D4F91E20FFF74D
:10A9E000EBFC86B2300AA0730420FFF7E5FC0006FA
:10A9F000000E0DD002206946087101AB0122122120
:10AA00002D2000F0BFF9A08B012109030843A0838A
:10AA100000F078F820600620FFF7CEFC6060072089
:10AA2000FFF7CAFCA060F006C00E207501D110200F
:10AA30002075C0B200F0E2F9E80707D0FFF7A3FCE9
:10AA4000A08B0121C9020843A0830AE0052136201A
:10AA500000F02EF81549084002460521362000F086
:10AA600077F90120FFF734FC0021042000F036F8CC
:10AA7000A0610021262000F031F815218903084348
:10AA800002460021262000F06EF900222621362001
:10AA900000F05EF900F036F8206000207CBD000078
:10AAA000F40000203001CADE00000020FFFD00009D
:10AAB00038B5094C89B280B26B46022200F028F802
:10AAC000002806D1684640780102684600780818D8
:10AAD00084B2204638BD0000FFFF000038B50024D6
:10AAE000E44389B280B26B46042200F011F80028DA
:10AAF00006D103216846435C2202D418491EFAD5C8
:10AB0000204638BD10B500210846FFF7E7FF10BD0D
:10AB100038B5002909D0402420436C462070C8B2C3
:10AB20007F2906D8607002200AE06946087001207B
:10AB300006E0802420436C466070C809A0700320A2
:10AB4000694600F095FA38BD10B5144603460A462A
:10AB500021461120FFF7DCFF10BD10B5034605228A
:10AB600000211520FFF7D4FF10BD10B501210620EC
:10AB7000FFF7B4FF10BD10B50346052200211720D2
:10AB8000FFF7C6FF10BD38B50546002069460870BE
:10AB900000F0C4F8FF2401342246002D01D0032226
:10ABA000120200210D2000F0D3F8002D13D06B46C7
:10ABB000012203210F20FFF7ABFF68460078000752
:10ABC00009D5FFF7A9FE224600210D2000F0C0F8AC
:10ABD0000020C04338BD002038BD10B50246012119
:10ABE0000A2000F0C0F810BD10B5044600211A205C
:10ABF000FFF774FF000D22030005120B0243002132
:10AC00001A2000F0B0F810BD10B5024602492E20FF
:10AC100000F09EF810BD000004180000F8B50546CD
:10AC20006B46012203210420FFF772FF0126114C1D
:10AC30003607002D0DD02A4600210C2000F088F8A0
:10AC4000694608781021084369460870A0693043B6
:10AC500007E069460878EF21084069460870A06956
:10AC6000B0430B46A06101220321042000F08AF8C2
:10AC7000F8BD0000F400002010B5024600211820A5
:10AC800000F066F810BD0000F8B5074600256846DC
:10AC90000570B807204C2E4600280ADA8020694645
:10ACA00008706B46012200210D2000F06BF8012096
:10ACB0002073F8076946087821D0062108436946C1
:10ACC00008706B46012200210D2000F05BF8032183
:10ACD0000F20FFF7EDFE8121C900084219D0402066
:10ACE000694608706B46012200210D2000F04AF8E9
:10ACF0000020FFF7FDFD00252673ED4309E002214A
:10AD00000843694608706B46012200210D2000F0BF
:10AD100039F82846F8BD0000140100201CB56B4628
:10AD2000012203210F20FFF7F3FE6846007840223E
:10AD3000C1091040C9014000814208D00120694684
:10AD40000871024601AB03210D2000F01BF81CBD69
:10AD500008B56B461A70120A5A7089B280B2022284
:10AD600000F010F808BD38B500236C46E254120A12
:10AD70005B1C042BFADB89B280B22346042200F06C
:10AD800001F838BD38B58024002909D0C0252843F2
:10AD90006D462870C8B27F2907D86870022009E084
:10ADA000204369460870012004E020436870C80908
:10ADB000A8700320694600F097F938BD10B5144615
:10ADC000012312189B029A4202D90020C04310BDF1
:10ADD0000B46821E21460920FFF7D4FF002010BD3C
:10ADE00010B5054A8905126901430A43002108206C
:10ADF000FFF7B9FF002010BDF400002038B504466D
:10AE00006B4601220E212B20FFF782FE6846007858
:10AE1000E10640094001C90E0143684601706B46D6
:10AE200001220E212B20FFF7ADFF38BD10B5002108
:10AE300042541C06120A22431B0A491C0429F7DB50
:10AE400010BD000013B501231A4669460248FDF7FC
:10AE500053FA00981CBD00002C150020FBF76EFF74
:10AE6000FEF742FCFDF7E8FD3E493F48002522C0C1
:10AE700005608561C5613D490562C1600838FCF720
:10AE8000A5F8FDF7C5FDFDF7A7FEFDF783FEFDF76D
:10AE90008BFD052601223607D1033046FBF739FF2B
:10AEA000FEF7D6FAFDF756FCFAF740FEFAF718FE61
:10AEB0000721B015FFF704FD2D4C0A21208A01223D
:10AEC0004843608311033046FBF723FF2648C8221E
:10AED00028498830FDF79AF9274F284EE078002856
:10AEE0003CD0FEF701FCE570FBF784F820700F28DA
:10AEF0000AD9012211033046FBF70BFFFEF774FC61
:10AF000000220121090309E0012251033046FBF729
:10AF100000FFFEF769FC0022012149033046FBF7E0
:10AF2000F8FEFDF765FB608B002801D0401E6083B2
:10AF30001348618B00780843D0D13878002801D0BD
:10AF40000328CBD10121C9023046FBF7D9FE0028E6
:10AF5000C4D101210846FCF753F9BFE7FDF748FBD0
:10AF6000BCE70000007C0040A4140020FFFF0000AC
:10AF7000BC000020580C00205A00002000040050A3
:10AF80003600002010B586B01748FBF77AFF142171
:10AF90006846FAF70CF9154800900320019000204C
:10AFA0000290052069460007FBF7B4FD694610488A
:10AFB000FBF7B0FD69460F48FBF7ACFD01210846E1
:10AFC000FCF71EF9FF2401342046FCF7EBF80A4990
:10AFD00008680422104308602046FCF7F5F8FCF7E7
:10AFE000FBF806B010BD0000A4140020FFFF000015
:10AFF00000040050000800500070004010B501220D
:10B00000920218491848FAF70BFE164817490288A9
:10B010008A4225D0018004218180FF21F531C18041
:10B020000A21018100211E224181D2438281012215
:10B03000C2810184018241828182C1820183818334
:10B040004323C38602230387782343878287C287EB
:10B0500002464032118451849184C18300F02EF85D
:10B0600010BD0000200D002000FC0008AA550000C3
:10B07000F0B58C4600251026052109078E620E4C7E
:10B0800008E067467F5DE760A768FF07FCD0E768D8
:10B090001F706D1C8542F4DB0020074606E0E76068
:10B0A000A568ED07FCD0E5681D54401C9042F6D31E
:10B0B0008E610020F0BD00000030014070B572B616
:10B0C0000124074DA40221462846FAF78FFD0028E7
:10B0D00004D0224603492846FAF778FE62B670BDCE
:10B0E00000FC0008200D0020F0B5002510260527E3
:10B0F0009C463F070B46BE620C4C06E0595DE16082
:10B10000A168C907FCD0E1686D1C8542F6DB002010
:10B1100007E06146095CE160A168C907FCD0E1680D
:10B12000401C9042F5D3BE610020F0BD00300140CC
:10B130000000010203040005405C0000A05C040064
:10B14000C06C0800805C0400E03F1E00E07D1E0033
:10B1500007A9022570889B880A00160001000600D6
:10B160000100020087008D002D001A3152001A33B1
:10B170009A001A351D011A376B003B31BE003B3374
:10B180005E013B3596023B37000099599959EB51C6
:10B190008F421E45142E0080EB51F5283333E13ADF
:10B1A000703DE13AC235852BC2353333C235C235E5
:10B1B000AE47E13A5138A33051380000000000009A
:10B1C0000000010203040607080900000000010254
:10B1D0000304030406080C1018203000FCB100081A
:10B1E00000000020F400000050A20008F0B20008A7
:10B1F000F40000206419000060A2000800070400A9
:10B20000091E080540082609104008560805400890
:10B21000261D040008BE1D040008BED8BC4010084E
:10B22000010000000000C842000000000000000013
:10B23000000000000000000000000000000000000E
:10B2400000000000010000000000000000000000FD
:10B2500000000000000000008C0A00000000000058
:10B2600000000000000000000000000000000000DE
:10B2700000000000000000000000000000000000CE
:10B2800000000000000000000000000000000000BE
:10B2900000000000000000000000000000000000AE
:10B2A00000000000020214000909000200810000F1
:10B2B000000000000100000000000000000000008D
:10B2C000000000000000000000000000000000007E
:10B2D000000000000000000000000000000000006E
:10B2E000000000000000000000002000000000003E
:04000005080050C1DE
:00000001FF
